:1000000011298030A100FE30AF200130AF207530C3
:10001000A7003030C628A101A117AF00AF08031D0B
:100020001328030114280130AF020310A20CA20C04
:10003000A20CC0302205403EAF07FE30AF202F0893
:10004000AF28A101A117AF00FE30AF202F08AF28C5
:10005000A401AA00AB01A01124080319A0150530C2
:10006000A3002730A900103041200330A900E83058
:100070004120A90164304120A9010A3041202A0809
:100080004828A8002B08A7002A08A600DA2026087E
:10009000A600A3030319A011240803195228230260
:1000A000031859282608031DA011A0195928303E0D
:1000B000AF280800A300240803190C292308AF2047
:1000C000A4035B28AD000611861183160611861164
:1000D0000F30860583122D08A0188C283E30A7000B
:1000E0008030C6203330AC00A0201330A700883009
:1000F000C620A0206430C520A0206430C520223056
:10010000AC00A02028308B200C308B2006308B20B8
:10011000A0142D088C282014AC00201C9A288611CD
:10012000033C031C9F289F200530A700DC30C6201D
:10013000031408002014FE3C0319AD288615201C6A
:10014000201006150F3086052C08F039860406119C
:10015000AC0E2018A0283230C5202D080C29A11B78
:10016000622883178001840AFF3E031DB2280C29F0
:10017000A901A800FF30A807031CA907031C0C292C
:100180000330A700DF30C620BA28A701E83EA6004A
:10019000A709FC30031CCF28A6070318CC28A60704
:1001A0000000A70FCC282618D528A61CD9280000A7
:1001B000D9280800AB01AA011030AC00270DAA0D08
:1001C000AB0D2808AA022908031C290FAB0203184B
:1001D000F0282808AA0729080318290FAB070310DD
:1001E000A60DA70DAC0BDE2826080C291030B00098
:1001F000A701A601AD0CAC0C031C04292808A60716
:1002000029080318290FA707A70CA60CAB0CAA0CEA
:10021000B00BFA282A080C29831383120313000059
:100220000800A00107309F00E03083168500FF30F2
:10023000860081138312850186012030840060309E
:10024000B220A03084005030B22020308400303002
:10025000B120C830B82001207730622062206220AF
:100260002E3062207030622069306220633062205C
:100270006230622061306220733062206930622017
:10028000633062202E3062206E3062206C3062203B
:100290000B30A900B830B92001204430622043302F
:1002A0006220463062203230622030306220553089
:1002B00062204B3062204430622020306220622075
:1002C000563062202D306220323062200730A90083
:1002D000D030B920012041306220643062206A3081
:1002E00062207530622073306220743062202030CA
:1002F00062204C30622044306220523062208618E6
:100300008729851F85290514862905107F29012045
:10031000533062206530622061306220723062208A
:1003200063306220683062202030622073306220A7
:1003300069306220673062206E3062206130622056
:100340006C306220361405128316051283123D2A82
:10035000C3013C03A500C90149082502031CC129AA
:10036000E421B61CBF294308A6004908A200A60143
:10037000A20A0314A60DA20BBA292608C304C90FAA
:10038000AC29B2014308B100B20CB10CB20CB10CF3
:10039000B20CB10CB20CB10C0F30B2053208AD008A
:1003A0003108AC00A9010A30A800F620B1002B08E2
:1003B000B200B4014308B3000F30B3050030B405F8
:1003C00031083307C3000800BA01B9010618F9293A
:1003D0000130B820B90A0319BA0A0B303A02031CDB
:1003E000F829031DF729B9303902031CF829922D89
:1003F000E6299B30B8200618B614061CB610361C29
:100400001D2AAD014408AC00A9011430A800F62053
:10041000B1002B08B2003208A7003108A600A901DC
:100420003A30A800DA20BD008030A1000230A200DE
:100430003D080D20FF306220302A8030A1000130BD
:10044000A2003D080D200230A40044082920030129
:100450003619013EB618013A03193611031D361537
:10046000C40A85140130A900F430B9208510A9010F
:10047000F030A8002808B9200800BB01C4013612DA
:10048000361ADD2ABA01B901061C572AB90A03191E
:10049000BA0A0130B820AF303A02031C562A031DB5
:1004A000552AC9303902031C562A922D442ABA0112
:1004B000B9010618932AB90A0319BA0A0A30B820F2
:1004C0003618872A39080B3A3A04031D722A8030FD
:1004D000A1000130A2003D080D20353062203930E6
:1004E0006220862A3908193A3A04031D792A8514AC
:1004F000862A39084B3A3A04031D802A8510862A39
:100500003908FA3A3A04031D862A922D922A1130AC
:100510003A02031C922A031D912A95303902031CCA
:10052000922A922D592A41303B02031C982A922D7F
:10053000BB0A3A08031DA02A65303902031CA12A10
:100540003616361CDC2AAD013B08AC00A90114307C
:10055000A800F620B1002B08B2003208A70031082D
:10056000A600A9014130A800DA20BD008030A1001A
:1005700080302120463062206F306220753062204A
:100580006E3062206430622020306220733062203E
:1005900069306220673062206E30622061306220F4
:1005A0006C306220203062208030A1000230A20036
:1005B0003D080D20FF306220402A361C012B01200F
:1005C000493062206E3062206930622074306220CF
:1005D00069306220613062206C30622069306220B4
:1005E0007A306220653062202E30622062206220E4
:1005F0008030A100C03021201430A4005F305A2088
:10060000702B0B30BD000130A2003D080B20A10172
:10061000B61D192B3B3041020318102BC10A182BB1
:10062000C101173045020318172BC50A182BC50145
:100630001D2B4208C1004608C500051B2D2B45088F
:10064000031D252B0C30C7002C2B0D304502031C3D
:100650002C2B0C304502C700322B4508C700203038
:10066000622062200A3047020318382B20306220B3
:100670008030A100470828203A3062200230A400D0
:10068000410829203A306220303062206220051B68
:10069000592B0C3045020318522B613062206D300B
:1006A0006220562B703062206D3062201130BD0008
:1006B0005B2B1330BD00410803190130031D0301FA
:1006C000B5001E30410203190130031D030135043A
:1006D000B50001308618030135040319702B6A2D0B
:1006E000361E682DE4210130C9000F30490203187D
:1006F0007C2BE421C90F752B3611B611E421E421BE
:10070000E421B61C852B0514862B05101230C90078
:100710001430490203188F2BE421C90F882BE421E0
:100720000730BC00A8214308C200E421361D992BE4
:10073000B6150630BC00A8214308C600E421361DCA
:10074000A22BB6150630BC00A8214308BE0003301A
:10075000BC00A8214308C8000530BC00A8214308FC
:10076000C0000830BC00A8214308BF00E421361DAA
:10077000BA2BB615361CC02BB619BF2B361001206C
:10078000B619672D8030A100803021200930A400E7
:1007900020305A208030A100C03021201430A40025
:1007A00020305A2080302120A10101304802031D51
:1007B000E62B4D3062206F3062206E306220643054
:1007C000622061306220793062205B2C0230480266
:1007D000031DF92B54306220753062206530622091
:1007E0007330622064306220613062207930622090
:1007F0005B2C03304802031D102C573062206530FB
:100800006220643062206E30622065306220733076
:1008100062206430622061306220793062205B2C7B
:1008200004304802031D252C5430622068306220B9
:100830007530622072306220733062206430622032
:1008400061306220793062205B2C05304802031D44
:10085000362C46306220723062206930622064306B
:10086000622061306220793062205B2C06304802C1
:10087000031D4B2C533062206130622074306220A3
:1008800075306220723062206430622061306220F4
:10089000793062205B2C07304802031D5B2C5330FB
:1008A0006220753062206E306220643062206130D8
:1008B0006220793062208030A100C03021203E08C3
:1008C00028202030622001304002031D762C4A305F
:1008D0006220613062206E306220753062206130AB
:1008E00062207230622079306220322D0230400264
:1008F000031D8B2C463062206530622062306220FE
:100900007230622075306220613062207230622065
:1009100079306220322D03304002031D9A2C4D3075
:100920006220613062207230622063306220683061
:100930006220322D04304002031DA92C4130622078
:100940007030622072306220693062206C30622028
:10095000322D05304002031DB42C4D306220613031
:10096000622079306220322D06304002031DC12CF6
:100970004A306220753062206E306220653062201D
:10098000322D07304002031DCE2C4A3062207530D4
:1009900062206C30622079306220322D08304002B3
:1009A000031DDF2C413062207530622067306220E9
:1009B000753062207330622074306220322D09302D
:1009C0004002031DF62C53306220653062207030E7
:1009D000622074306220653062206D3062206230A7
:1009E00062206530622072306220322D0A3040026F
:1009F000031D092D4F306220633062207430622065
:100A00006F30622062306220653062207230622076
:100A1000322D0B304002031D1E2D4E3062206F30F0
:100A2000622076306220653062206D306220623054
:100A300062206530622072306220322D0C3040021C
:100A4000031D322D44306220653062206330622005
:100A5000653062206D306220623062206530622035
:100A600072306220203062203230622030306220CA
:100A70008030A1000230A4003F0829200930400244
:100A8000031D512D1430C9000230A20049080B206B
:100A9000A101051C4E2D53306220502D573062208D
:100AA000672D1230C9000230A20049080B20A101B5
:100AB000051C612D2A306220533062202A306220CA
:100AC000672D2A306220573062202A306220692D3B
:100AD000922D3D2A851F712D051283160512831252
:100AE000732D8316051683129B30B8204108031915
:100AF0000130031D0301B5000130861803013504E0
:100B00000319832D0515851585140130A900F430CE
:100B1000B9200511851185100130A9004A30B9208E
:100B2000C40A732B01204E3062206F3062202030C7
:100B300062207330622069306220673062206E303C
:100B40006220613062206C3062202030840060308E
:100B5000B220A03084005030B220203084003030E9
:100B6000B1200618B616061CB61203010618013E7F
:100B7000B61A013C031DC22DB70A0319B80A013089
:100B8000B820B52D0301B61A0130013A0319B61287
:100B9000031DB61603010618013EB61A013C031DDB
:100BA000D72DB70A0319B80A0130B820CA2D03306F
:100BB0003802DE30031937020318A52D36143D2AFA
:02400E00503F21
:00000001FF
